:100000000C945D000C9485000C9485000C94850084
:100010000C9485000C9485000C9485000C9485004C
:100020000C9485000C9485000C9485000C9485003C
:100030000C9485000C9485000C9485000C9485002C
:100040000C94E2030C9485000C94B0030C948A0386
:100050000C9485000C9485000C9485000C9485000C
:100060000C9485000C9485000000000025002800F9
:100070002B0000000008000201000003040700003C
:1000800000000000000000000000240027002A00FB
:10009000010204081020408001020408102001021F
:1000A00004081020040404040404040402020202EC
:1000B00002020303030303035A0811241FBECFEFF8
:1000C000D8E0DEBFCDBF11E0A0E0B1E0E8E2F1E1B1
:1000D00002C005900D92AC31B107D9F722E0ACE136
:1000E000B1E001C01D92A33EB207E1F710E0CDE5FB
:1000F000D0E004C02197FE010E948708CC35D107CB
:10010000C9F70E942C040C9492080C940000E09112
:100110004602F09147020190F081E02D682F86E4BD
:1001200092E00994CF92DF92EF92FF920F931F9388
:10013000CF93DF936C017A018B01C0E0D0E0CE1544
:10014000DF0589F0D8016D918D01D601ED91FC910B
:100150000190F081E02DC6010995892B11F47E01F3
:1001600002C02196ECCFC701DF91CF911F910F9173
:10017000FF90EF90DF90CF900895089580E090E099
:100180000895FC01538D448D252F30E0842F90E09D
:10019000821B930B541710F0CF9608950197089582
:1001A000FC01918D828D981761F0828DDF01A80F7F
:1001B000B11D5D968C91928D9F5F9F73928F90E0A1
:1001C00008958FEF9FEF0895FC01918D828D981710
:1001D00031F0828DE80FF11D858D90E008958FEF4D
:1001E0009FEF0895FC01918D228D892F90E0805C16
:1001F0009F4F821B91098F739927089586E492E09F
:100200000E94F20021E0892B09F420E0822F08955A
:10021000FC01848DDF01A80FB11DA35ABF4F2C91A3
:10022000848D90E001968F739927848FA689B78972
:100230002C93A089B1898C9180648C93938D848D4B
:10024000981306C00288F389E02D80818F7D80831A
:100250000895EF92FF920F931F93CF93DF93EC01DA
:1002600081E0888F9B8D8C8D981305C0E889F98972
:10027000808185FD24C0F62E0B8D10E00F5F1F4F8F
:100280000F731127E02E8C8DE8120CC00FB607FCFF
:10029000FACFE889F989808185FFF5CFCE010E94E8
:1002A0000801F1CF8B8DFE01E80FF11DE35AFF4FDE
:1002B000F0820B8FEA89FB898081806207C0EE891A
:1002C000FF896083E889F98980818064808381E087
:1002D00090E0DF91CF911F910F91FF90EF900895E3
:1002E000CF93DF93EC01888D8823C9F0EA89FB89DD
:1002F000808185FD05C0A889B9898C9186FD0FC0D4
:100300000FB607FCF5CF808185FFF2CFA889B989A8
:100310008C9185FFEDCFCE010E940801E7CFDF91E0
:10032000CF91089580E090E0892B29F00E94FE0093
:1003300081110C940000089590E0FC01EE58FF4FED
:100340003491FC01E057FF4F2491FC01EC55FF4F25
:10035000E491EE2309F43BC0332339F1333091F0BB
:1003600038F43130A9F0323001F584B58F7D12C0F8
:10037000373091F03830A1F03430B9F480918000FA
:100380008F7D03C0809180008F77809380000DC0A7
:1003900084B58F7784BD09C08091B0008F7703C08A
:1003A0008091B0008F7D8093B000F0E0EE0FFF1FD2
:1003B000E859FF4FA591B4918FB7F894EC91611172
:1003C00003C020952E2301C02E2B2C938FBF0895A0
:1003D000CF93DF9390E0FC01E057FF4F2491FC01A5
:1003E000EC55FF4F8491882361F190E0880F991FAD
:1003F000FC01EA57FF4FC591D491FC01E859FF4F2A
:10040000A591B491611109C09FB7F8948881209596
:1004100082238883EC912E230BC0623061F49FB756
:10042000F8943881822F809583238883EC912E2B3A
:100430002C939FBF06C08FB7F894E8812E2B28839A
:100440008FBFDF91CF9108953FB7F89480911D0140
:1004500090911E01A0911F01B091200126B5A89B8B
:1004600005C02F3F19F00196A11DB11D3FBFBA2F46
:10047000A92F982F8827820F911DA11DB11DBC01A6
:10048000CD0142E0660F771F881F991F4A95D1F76B
:1004900008958F929F92AF92BF92CF92DF92EF9288
:1004A000FF926B017C010E9424024B015C01C1148C
:1004B000D104E104F104F1F00E942402DC01CB013B
:1004C00088199909AA09BB09883E9340A105B1057D
:1004D00070F321E0C21AD108E108F10888EE880E15
:1004E00083E0981EA11CB11CC114D104E104F104E5
:1004F00019F7DDCFFF90EF90DF90CF90BF90AF90D6
:100500009F908F9008951F93CF93DF93182FC3E090
:10051000D0E061E0812F0E949C016EE170E080E0FC
:1005200090E00E94490260E0812F0E949C016EE1F0
:1005300070E080E090E00E944902219751F7DF913E
:10054000CF911F910895209135013091360180910E
:100550004002909141022032310511F4807F0895CC
:100560002034310511F4807E08952038310511F4CE
:10057000807C08952115314009F48078089586E43F
:1005800092E00E94F200892BD1F386E492E00E946F
:10059000D0000895CF93C82F0E94BF02803241F44B
:1005A00084E10E9487008C2F0E94870080E10AC0AE
:1005B000809142029091430201969093430280936E
:1005C000420285E1CF910C9487000E94BF028032E5
:1005D00029F484E10E94870080E10AC080914202F0
:1005E000909143020196909343028093420285E1E9
:1005F0000C9487000F931F93CF93DF938C01CDE36F
:10060000D1E0CE018D5391408017910724F40E94D0
:10061000BF028993F6CFDF91CF911F910F9108957B
:100620008EBD00000DB407FEFDCF8EB50895CF93AB
:10063000DF9300D01F92CDB7DEB72B834A83698347
:100640000E9410036981862F0E9410034A81842F23
:100650000E9410032B81822F0F900F900F90DF913B
:10066000CF910C941003EF92FF920F931F93CF93AF
:10067000DF93EC018B01CB010E94FA0260E085E080
:100680000E949C018DE3E82E81E0F82E0C0F1D1FC7
:10069000C017D10781F0F70121917F014C2F6D2FF9
:1006A00080EC0E9417036DE270E080E090E00E9411
:1006B00049022196EDCF61E085E00E949C0180E136
:1006C000DF91CF911F910F91FF90EF900895CF93FD
:1006D000DF9300D0CDB7DEB7482F60E085E04983D7
:1006E0009A830E949C0120E049819A81692F8CE4C1
:1006F0000E9417036EE170E080E090E00E944902E2
:1007000061E085E00F900F90DF91CF910C949C01F8
:100710000E948D081F920F920FB60F9211242F93F3
:100720003F934F935F936F937F938F939F93AF9379
:10073000BF93EF93FF9386E492E00E940801FF913C
:10074000EF91BF91AF919F918F917F916F915F9149
:100750004F913F912F910F900FBE0F901F901895C2
:100760001F920F920FB60F9211242F938F939F9386
:10077000EF93FF93E0915602F09157028081E09150
:100780005C02F0915D0282FD12C0908180915F0257
:100790008F5F8F7320916002821751F0E0915F02AA
:1007A000F0E0EA5BFD4F958F80935F0201C080818E
:1007B000FF91EF919F918F912F910F900FBE0F900E
:1007C0001F9018951F920F920FB60F9211242F931E
:1007D0003F938F939F93AF93BF938091210190910B
:1007E0002201A0912301B091240130911C0123E04A
:1007F000230F2D3720F40196A11DB11D05C026E859
:10080000230F0296A11DB11D20931C01809321018D
:1008100090932201A0932301B093240180911D01A4
:1008200090911E01A0911F01B09120010196A11D80
:10083000B11D80931D0190931E01A0931F01B093E1
:100840002001BF91AF919F918F913F912F910F9078
:100850000FBE0F901F901895789484B5826084BD68
:1008600084B5816084BD85B5826085BD85B58160B4
:1008700085BD80916E00816080936E001092810032
:1008800080918100826080938100809181008160ED
:1008900080938100809180008160809380008091AE
:1008A000B10084608093B1008091B000816080933A
:1008B000B00080917A00846080937A0080917A0001
:1008C000826080937A0080917A00816080937A00C0
:1008D00080917A00806880937A001092C100E09144
:1008E0005602F091570282E08083E0915202F0912B
:1008F00053021082E0915402F091550287E6808302
:1009000010925E02E0915A02F0915B0286E08083D1
:10091000E0915802F0915902808180618083E091DA
:100920005802F0915902808188608083E0915802DA
:10093000F0915902808180688083E0915802F091A3
:10094000590280818F7D808361E085E00E94E8010B
:1009500085E090E00E94830261E086E00E94E80169
:1009600086E090E00E94830261E087E00E94E80157
:1009700087E090E00E94830219E7212E10E0312EDB
:100980000BE8C02EDD24D394AA24A394B12C9EEAB4
:10099000492E90E0592E2AE9822E20E0922E809155
:1009A000440290914502892B11F061E001C060E0A2
:1009B00085E00E949C018091420290914302892B24
:1009C00011F061E001C060E086E00E949C012FB759
:1009D000F8948091210190912201A0912301B0917E
:1009E00024012FBF409125015091260160912701DC
:1009F000709128018C019D01041B150B260B370BF0
:100A0000083211052105310508F46BC080932501DA
:100A100090932601A0932701B0932801C091010172
:100A200080EE8C0F813A28F08091000181958093AF
:100A3000000180910001C80FC09301010C2F10E04C
:100A400061E087E00E94E801C11102C060E003C0DC
:100A5000CF3F29F461E087E00E949C0142C0F10190
:100A600084918330F9F048F48130B9F08230A1F5F7
:100A700084B5806284BDC8BD34C08730E9F0883059
:100A800019F1843049F58091800080628093800064
:100A900010938B0000938A0024C084B5806884BDC5
:100AA000C7BD1FC080918000806880938000109334
:100AB00089000093880015C08091B0008068809301
:100AC000B000C093B3000DC08091B00080628093ED
:100AD000B000C093B40005C0003811050CF0BACFC7
:100AE000B5CF86E492E00E94F200892B09F4DFC2C0
:100AF0000E94BF02813509F46CC2B0F4813409F45C
:100B000051C040F48033C1F18133D9F1803209F012
:100B1000BCC2B1C2853409F4DDC0803509F4DFC040
:100B2000823409F0B2C253C0813609F45BC1D0F4FB
:100B3000863509F43DC2803609F452C1853509F085
:100B4000A4C20E94BF02C82F0E94BF02282F30E01B
:100B5000322F2227C9018C0F911D9093410280935F
:100B6000400265C2843709F4CAC1853709F462C2FC
:100B7000843609F08AC239C11092430210924202AF
:100B800056C20E94BF02803209F075C284E10E9401
:100B9000870047E050E064E171E086E492E00E9463
:100BA000920067C20E94BF02813859F020F4803859
:100BB00061F482E00BC2823831F0833931F483E58D
:100BC00005C281E003C282E101C280E0FFC184E18D
:100BD00090E00E94FA0220913D0120932A01809129
:100BE0003E0180932B0180913F0180932C018091E5
:100BF000400180932D018091410180932E018091CD
:100C0000420180932F0180914301809330018091B4
:100C1000440180933101809145018093320180919C
:100C2000470190E0982F882730914801830F911D4C
:100C300090933401809333018091490190E0982F83
:100C4000882730914A01830F911D9093360180933C
:100C5000350180914B0190E0982F882730914C010D
:100C6000830F911D909338018093370180914D013E
:100C700090E0A0E0B0E0BA2FA92F982F88273091FC
:100C80004E01830F911DA11DB11DDC0199278827FD
:100C900040914F0150E0542F4427052E000C660B65
:100CA000770B840F951FA61FB71F30915001830F3C
:100CB000911DA11DB11D8093390190933A01A0931C
:100CC0003B01B0933C0181E0203E08F480E080933A
:100CD0003F02ADC185E090E00E94FA02A8C1809178
:100CE000440290914502892B09F0A1C160913F0215
:100CF0008AE00E949C0161E08AE00E94E801CFB78F
:100D0000F89480913E02811125C0F2018491F40192
:100D10009491E82FF0E0EE0FFF1FEA57FF4FA591E7
:100D2000B4918C91982321F461E08AE00E949C01A7
:100D300061E08AE00E94E8018CB580618CBD8CB5D1
:100D400080648CBD61E08DE00E94E80161E08BE091
:100D50000E94E80180913E028F5F80933E02CFBFE8
:100D600080913D02882379F08FB7F89490913D02ED
:100D7000913039F49DB3909329019DB39DBB8FBFF2
:100D800002C08093290183E58CBD1DBC60E08DE02D
:100D90000E949C0164E170E080E090E00E944902C2
:100DA000C0913F0281E06C2F68278AE00E949C017D
:100DB000C6010197F1F76C2F8AE00E949C0162E363
:100DC00070E080E090E00E94490220E040E063E5AE
:100DD0008CEA0E941703B0924502A092440227C1F8
:100DE0000E94BF020E94BF0222C10E94BF02C82F00
:100DF0000E94BF02D0E0DC2FCC27C80FD11D0E947B
:100E0000BF02863409F044C0CE010E94FA020E945B
:100E1000BF02803209F02FC184E10E9487000E9446
:100E2000A3028C01E12CF12CEC16FD066CF50E945E
:100E3000A3023C010817190731F0C8010E9467039B
:100E40000E94A3023C010091400210914102F7016F
:100E5000E35CFE4F2081402F612F80E40E94170346
:100E6000F2E0EF0EF11CF701E45CFE4F2081402F11
:100E7000612F88E40E9417030F5F1F4F10934102F8
:100E8000009340028301D0CFC8010E946703F1C0E4
:100E9000853409F08BC0009140021091410280918D
:100EA0003701909138018C179D0718F0000F111F22
:100EB0000BC08091420290914302019690934302AD
:100EC00080934202C1E111C0C132D10548F060E215
:100ED00070E0C8010E943303005E1F4FA097F4CF5B
:100EE000BE01C8010E943303C0E10E94BF028032EC
:100EF00009F0C1C084E10E9487008C2FD6C00E94F7
:100F0000BF02C82F0E94BF02082F0E94BF02182FE5
:100F10000E94BF02803209F0AEC0D0E0DC2FCC27A7
:100F2000C00FD11D84E10E948700163431F500E026
:100F300010E00C171D070CF09CC04091400260911E
:100F4000410220E080E20E9417030E948700409146
:100F500040026091410220E088E20E9417030E9453
:100F60008700809140029091410201969093410246
:100F7000809340020E5F1F4FDCCF1534B9F400910F
:100F8000400210914102000F111FC00FD11F0C171A
:100F90001D0709F46EC02FEF402F612F80EA0E94D9
:100FA00017030E9487000F5F1F4FF1CF81E17DC0C3
:100FB00084E090E00E94FA022091400140913F01BC
:100FC00060913E0180913D010E9417030E94CA0278
:100FD0006EC010924302109242029FB7F894809123
:100FE0003E02882319F0815080933E0280913E0298
:100FF000811105C08CB58F7B8CBD10923D029FBFC7
:1010000060E08BE00E94E80160E08DE00E94E80172
:1010100060913F0281E068278AE00E949C0160E0C5
:101020008AE00E94E80110924502109244020E9458
:10103000E5023DC00E94BF028032E9F484E10E94D3
:10104000870020E040E060E080E30E9417030E94F8
:10105000870020E041E060E080E30E9417030E94E7
:10106000870020E042E060E080E30E9417030E94D6
:10107000870080E11AC0809142029091430201965C
:1010800090934302809342020FC08091420290915C
:101090004302019690934302809342020E94BF0252
:1010A000803211F482E101C085E10E9487000E9434
:1010B000920175CCE6E4F2E01382128288EE93E0AE
:1010C000A0E0B0E084839583A683B78386E091E0B7
:1010D0009183808385EC90E09587848784EC90E011
:1010E0009787868780EC90E0918B808B81EC90E0F5
:1010F000938B828B82EC90E0958B848B86EC90E0D6
:10110000978B868B118E128E138E148E0895EE0F90
:10111000FF1F0590F491E02D099481E090E0F89490
:081120000C949208F894FFCF33
:1011280008800000000029019200C1007001F2004F
:0C113800D000E400415652204953500002
:00000001FF
